:020000040000FA
:040000006F303A28FB
:08000800A000030EA100831209
:1000100005191128831601178312B2308100B0012F
:100020002C2883160113831203140B190310A80D37
:10003000A90DAA0DAB0DAC0DAC16FF302C02031DA3
:100040002C28FA302B02031D2C2831152A08AF006A
:100050002908AE002808AD008B100B11210E83007B
:06006000A00E200E0900B5
:0C007400203084008001840A80300402E7
:10008000031C3C28622183160C30850587018312EE
:10009000850187010730990000309A0010308316DF
:1000A0008E008312603083168F0083120030831617
:1000B00091009F008312C830831681008312313073
:1000C0009000003083168C00831210308B00A0212A
:1000D00081018E018F010B118B100B108C018B177E
:1000E000802031198C204421B30B7E280310851900
:1000F0000314B90DF03039020319ED20A121702845
:1001000064003210B00A301F8B28AC01AB01AA0189
:10011000A901A801B001080031110130B7008B130B
:100120002030370783169B001C141A088312A40082
:100130001030370783169B001C141A088312A30083
:10014000A6000230A6060030370783169B001C1459
:100150001A088312A200A7000130A7068B17321CD1
:10016000B72822090339A200A309A409A509240874
:100170002F02031DE72823082E02031DE72822086B
:100180002D02031DE72801303702031DCC283D183E
:10019000CC283D143E147D2102303702031DD528A2
:1001A000BD18D528BD143E14862103303702031D27
:1001B000DE283D19DE283D153E148F21043037021C
:1001C000031DE728BD19E728BD153E149821B70A7D
:1001D00005303702031808008F280130B600B3003D
:1001E000B400B500B70085018701B1138020B30BBF
:1001F0001329031085190314B90DF03039020319BE
:100200003A29B41F8501B41F8701B40B132937089D
:10021000B6080319B60003191129FF3085008700BD
:10022000B6039630B400311DF6283111321C1D2959
:100230002D090339AD00AE09AF092F1CF6288E0138
:100240008F010C1CF6280C102E1EF6288B13203064
:100250003707BB002F08BA004D2110303707BB000D
:100260002E08BA004D2100303707BB002D08BA0018
:100270004D218B1785018701B70AB601053037027A
:10028000031CF628A02108003E1C08003E10103078
:10029000BB003D08BA004D2108008B133A088316B5
:1002A0001C159A0083123B0883169B0055309D0055
:1002B000AA309D009C1464009C185B291C118312B9
:1002C0008B170800831610309B001C141A08831229
:1002D000BD00831620309B001C141A088312C20034
:1002E0000130C21BC200C2080319C2000130D50090
:1002F000D200EE30D000D10008000130D500D2008D
:10030000EE30D000D1000130BD0008000130D50032
:10031000D200EE30D000D1000230BD000800013024
:10032000D500D200EE30D000D1000430BD0008006E
:100330000130D500D200EE30D000D100BD01080060
:1003400008008F08031908008F01C10B080042083C
:10035000C100D50B08005608D50007303D0503192C
:10036000D829D21BD00AD21FD0030A305002031C56
:10037000D329D0010930D21FD0005203D2007F39D7
:10038000031DD329D10A10305102031CC829D10101
:100390005022D2006022D4007022D600D500D001B5
:1003A0000930D21FD00000238500242387000800D5
:0603B00085018701080031
:1004A00002308A0051083D1C572A883E8200BD1C3C
:1004B0005B2A883E82003D1D5F2A983E8200003400
:1004C00002308A0051083D1C672AA83E8200BD1CEC
:1004D0006B2AB83E82003D1D6F2AB83E8200003470
:1004E00002308A0051083D1C772AC83E8200BD1C9C
:1004F0007B2AD83E82003D1D7F2AE83E82000134DF
:100510000734873407348734033483340334833413
:100520000B3403340F3407340B34033403340734EF
:10053000053487340734253483340334073489344D
:100540000B3403348F3405348B34113403340334C7
:1005500001340134023402340434043408340834DD
:10056000103410342034203440344034803480340B
:10057000083404340234803440348034103402347B
:10058000043410342034013404344034843480344E
:10059000093409340A340A34083408340834083475
:1005A0000834183408341834083418341034083433
:1005B000093429340A341A34283408340834083405
:1005C0000A34383408341A3408345834103448346F
:1005D000293409340A340A342834083408344834B5
:1005E0002834183488341834283418341034083433
:1006000003308A005008541C072B4B3E8200D41C38
:100610000B2B563E8200541D0F2B613E8200D41DD1
:10062000132B6C3E8200541E172B773E8200D41E83
:100630001B2B823E8200541F1F2B8D3E8200D41F35
:10064000232B983E8200003403308A005008541C4B
:100650002B2BA33E8200D41C2F2BAE3E8200541DB8
:10066000332BB93E8200D41D372BC43E8200541E6A
:100670003B2BCF3E8200D41E3F2BDA3E8200541F1C
:10068000432BE53E8200D41F472BF03E820000340E
:0A0696001034203401340234003423
:0A06A000003400340034003400344C
:0406AC0010343034A2
:1006B0003134333433343334333433343334333404
:0E06C2000034003400340034003400340234BC
:0606D0000334233433342F
:0806D800103420340134023417
:0C06E000003410342034013402340034A3
:0206EE001034C6
:1006F0002034013402340034003402340134203414
:020700001034B3
:0C070400103430343134333433343334A7
:080710003134303410340034A0
:06071A00333423340334E4
:0E072000023400340034023403342334333402
:10073000333400343334003433340034333400344D
:04074000333400341A
:0A07460000340034003400340234A3
:0A075000043401342034103408345E
:04075C000034003431
:1007600000340034023406340734273437343F343D
:0E07720008341834383439343D343F343F34C1
:060780003F343F343F341A
:08078800043401342034103464
:0C0790000A3404340134203410340A34DC
:02079E0008341D
:1007A000103420340134063406340134203410343B
:0207B00008340B
:0C07B40008341834383439343F343934F8
:0807C000383418340834003409
:0607CA003F3437342734F0
:0E07D0000734063406340734273437343F34F8
:1007E0003F3400343F3400343F3400343F3400346D
:0407F0003F3400345E
:084000000C000300060006009D
:02400E00CC33B1
:10420000010078007A007C007E007B0079007F004E
:104210007D007A0078007E007C00FF00FF00FF0038
:104220000000F200F600FA00FE00F200F600FA00CC
:10423000FE00F200F600FA00FE00FF00FF00FF00A3
:10424000010005000500050005000900090009003E
:1042500009000D000D000D000D00FF00FF00FF0024
:10426000FF00FF00FF00FF00FF00FF00FF00FF0056
:10427000FF00FF00FF00FF00FF00FF00FF00FF0046
:10428000FF00FF00FF00FF00FF00FF00FF00FF0036
:10429000FF00FF00FF00FF00FF00FF00FF00FF0026
:1042A000FF00FF00FF00FF00FF00FF00FF00FF0016
:1042B000FF00FF00FF00FF00FF00FF00FF00FF0006
:1042C000FF00FF00FF00FF00FF00FF00FF00FF00F6
:1042D000FF00FF00FF00FF00FF00FF00FF00FF00E6
:1042E000FF00FF00FF00FF00FF00FF00FF00FF00D6
:1042F000FF00FF00FF00FF00FF00FF00FF00DD00E8
:00000001FF
